:04100000BBEF3FF013
:107F76000001BEEF3FF0000E926E000E956E010EF0
:107F8600C26EC250C30B0409C26E0D0EC16E000E46
:107F9600C06E000E946E000E826ECB68070ECA6E1F
:107FA6003C0EBD6E3C0EBA6EC28224D0C344E84677
:107FB600030B8C6EC4CFBEFFC3CF01F0060E026E5C
:107FC600D8900132022EFCD7013ABD500118CF0BD2
:107FD6000118BD6EC4CFBBFFC3CF01F0060E026E03
:107FE600D8900132022EFCD7013ABA500118CF0BB5
:0A7FF6000118BA6EC2A2D8D7D9D77D
:020000040020DA
:08000000FFFFFFFFFFFFFFFF00
:020000040030CA
:0E000000240E3F1EFF8181FF0FC00FE00F4056
:00000001FF
